:020000040000FA
:040800005FEF09F0AD
:1008100003B283EF05F0F2B4A1EF05F09EB0A9EFAB
:1008200005F09EB2B1EF05F0F2A81AEF04F0F2B2B3
:1008300032EF04F09EB61FEF04F00EEF09F09E9623
:1008400000011350000A06E000011350010A06E0FF
:100850000EEF09F0CAEC1EF00EEF09F0BEEC20F02E
:100860000EEF09F0CD90F2929EA03CEF04F0010152
:10087000533F3CEF04F0542BAEC1B2F1AFC1B3F122
:10088000B0C1B4F1B1C1B5F1AAC1AEF1ABC1AFF124
:10089000ACC1B0F1ADC1B1F1A6C1AAF1A7C1ABF134
:1008A000A8C1ACF1A9C1ADF1A2C1A6F1A3C1A7F144
:1008B000A4C1A8F1A5C1A9F19EC1A2F19FC1A3F154
:1008C000A0C1A4F1A1C1A5F19AC19EF19BC19FF164
:1008D0009CC1A0F19DC1A1F196C19AF197C19BF174
:1008E00098C19CF199C19DF1CECF96F1CFCF97F1F0
:1008F00053C198F154C199F1CF6ACE6A0101536B8B
:10090000546B9E90CD800FBC0F8E0FBA8BEF04F00E
:100910000F8A0EEF09F00F8C0FBEC7EF04F096C1DF
:100920009AF197C19BF198C19CF199C19DF19AC12F
:100930009EF19BC19FF19CC1A0F19DC1A1F19EC1FF
:10094000A2F19FC1A3F1A0C1A4F1A1C1A5F1A2C1CF
:10095000A6F1A3C1A7F1A4C1A8F1A5C1A9F1A6C19F
:10096000AAF1A7C1ABF1A8C1ACF1A9C1ADF1AAC16F
:10097000AEF1ABC1AFF1ACC1B0F1ADC1B1F1AEC13F
:10098000B2F1AFC1B3F1B0C1B4F1B1C1B5F1010180
:100990005E6B5F6B606B616B96515E2797515F2357
:1009A00098516023995161239A515E279B515F238F
:1009B0009C5160239D5161239E515E279F515F236F
:1009C000A0516023A1516123A2515E27A3515F234F
:1009D000A4516023A5516123A6515E27A7515F232F
:1009E000A8516023A9516123AA515E27AB515F230F
:1009F000AC516023AD516123AE515E27AF515F23EF
:100A0000B0516023B1516123B2515E27B3515F23CE
:100A1000B4516023B5516123D89001016133603333
:100A20005F335E33D8900101613360335F335E33EF
:100A3000D8900101613360335F335E3300C10CF144
:100A400001C10DF102C10EF103C10FF104C110F19A
:100A500005C111F106C112F107C113F108C114F16A
:100A600009C115F10AC116F10BC117F134C135F1F5
:100A700011B846EF05F00101620E046F010E056F1B
:100A8000000E066F000E076F4FEF05F00101A70E75
:100A9000046F020E056F000E066F000E076F5EC139
:100AA00000F15FC101F160C102F161C103F161ECCC
:100AB0001DF003BF04D018BE02D018A0108C11A0E6
:100AC00067EF05F010BA67EF05F00F80108A0CC1D0
:100AD00000F10DC101F10EC102F10FC103F110C10E
:100AE00004F111C105F112C106F113C107F114C1DE
:100AF00008F115C109F116C10AF117C10BF135C191
:100B000034F10EEF09F00392ABB2AB98AB8803015E
:100B100003EE00F080517F0BE92604C0EFFF802B2D
:100B20008151805D700BD8A48B8200008051815D63
:100B3000700BD8A48B9281518019D8B407900EEF16
:100B400009F0F2940101453F0EEF09F0462B0EEF3C
:100B500009F09E900101533F0EEF09F0542B0EEF68
:100B600009F09E9211B81EEF07F08BB4BFEF05F0AD
:100B700010ACBFEF05F08B84109CC0EF05F08B9498
:100B8000C3CF55F1C4CF56F1C28207B42AEF06F0A5
:100B900047C14BF148C14CF149C14DF14AC14EF139
:100BA0005EC162F15FC163F160C164F161C165F171
:100BB00096C1B6F197C1B7F198C1B8F199C1B9F131
:100BC0009AC1BAF19BC1BBF19CC1BCF19DC1BDF101
:100BD0009EC1BEF19FC1BFF1A0C1C0F1A1C1C1F1D1
:100BE000A2C1C2F1A3C1C3F1A4C1C4F1A5C1C5F1A1
:100BF000A6C1C6F1A7C1C7F1A8C1C8F1A9C1C9F171
:100C0000AAC1CAF1ABC1CBF1ACC1CCF1ADC1CDF140
:100C1000AEC1CEF1AFC1CFF1B0C1D0F1B1C1D1F110
:100C2000B2C1D2F1B3C1D3F1B4C1D4F1B5C1D5F1E0
:100C3000010155515B2756515C23E86A5D230E2E56
:100C40002AEF06F05CC157F15DC158F15B6B5C6B3C
:100C50005D6B078E0201002F0EEF09F03C0E006F56
:100C60001950E00BE00AE866128816AE108E00C13B
:100C70000CF101C10DF102C10EF103C10FF104C16C
:100C800010F105C111F106C112F107C113F108C13C
:100C900014F109C115F10AC116F10BC117F134C1E4
:100CA00035F101018A675CEF06F08B675CEF06F0B7
:100CB0008C675CEF06F08D6760EF06F090EF06F052
:100CC0008EC100F18FC101F190C102F191C103F118
:100CD0000101010E046F000E056F000E066F000E7D
:100CE000076F61EC1DF000C18EF101C18FF102C1EF
:100CF00090F103C191F1006785EF06F0016785EF80
:100D000006F0026785EF06F0036790EF06F08AC1F0
:100D10008EF18BC18FF18CC190F18DC191F10F805B
:100D2000D57ED5BE6DD0D6CF47F1D7CF48F145C1DE
:100D300049F1E86AE8CF4AF118BE02D018A0108C39
:100D4000109047C100F148C101F149C102F14AC107
:100D500003F101010A0E046F000E056F000E066F0D
:100D6000000E076F61EC1DF003AF1080010154A766
:100D7000C6EF06F00F9A0F9C0F9E0101000E5E6FEA
:100D8000600E5F6F3D0E606F080E616F010147BF1F
:100D9000D6EF06F04867D6EF06F04967D6EF06F0C3
:100DA0004A67D6EF06F0F288FBEF06F0F2985E6B2A
:100DB0005F6B606B616B966B976B986B996B9A6BC3
:100DC0009B6B9C6B9D6B9E6B9F6BA06BA16BA26BD7
:100DD000A36BA46BA56BA66BA76BA86BA96BAA6B87
:100DE000AB6BAC6BAD6BAE6BAF6BB06BB16BB26B37
:100DF000B36BB46BB56BD76AD66A0101456B466BB2
:100E00000CC100F10DC101F10EC102F10FC103F1DE
:100E100010C104F111C105F112C106F113C107F1AE
:100E200014C108F115C109F116C10AF117C10BF17E
:100E300035C134F10EEF09F00EEF09F00201002F79
:100E400075EF08F0D59ED6CF47F1D7CF48F145C111
:100E500049F1E86AE8CF4AF1D76AD66A0101456BE1
:100E6000466BD58E1950E00BE00AE866128817AE83
:100E7000108E16AE1B8C00C10CF101C10DF102C128
:100E80000EF103C10FF104C110F105C111F106C14A
:100E900012F107C113F108C114F109C115F10AC11A
:100EA00016F10BC117F134C135F10FA0109A11B82A
:100EB00065EF07F00101620E046F010E056F000E71
:100EC000066F000E076F6EEF07F00101A70E046FAB
:100ED000020E056F000E066F000E076F47C100F18E
:100EE00048C101F149C102F14AC103F161EC1DF0B1
:100EF00003BF81EF07F018BE02D018A0108C11B00C
:100F00000F800CC100F10DC101F10EC102F10FC142
:100F100003F110C104F111C105F112C106F113C1B1
:100F200007F114C108F115C109F116C10AF117C181
:100F30000BF135C134F102013C0E006F00C10CF120
:100F400001C10DF102C10EF103C10FF104C110F195
:100F500005C111F106C112F107C113F108C114F165
:100F600009C115F10AC116F10BC117F134C135F1F0
:100F700001018A67C3EF07F08B67C3EF07F08C6747
:100F8000C3EF07F08D67C7EF07F0F7EF07F08EC1EB
:100F900000F18FC101F190C102F191C103F1010192
:100FA000010E046F000E056F000E066F000E076F36
:100FB00061EC1DF000C18EF101C18FF102C190F111
:100FC00003C191F10067ECEF07F00167ECEF07F068
:100FD0000267ECEF07F00367F7EF07F08AC18EF1C5
:100FE0008BC18FF18CC190F18DC191F10F80109068
:100FF00047C100F148C101F149C102F14AC103F101
:1010000001010A0E046F000E056F000E066F000E40
:10101000076F61EC1DF003AF1080010154A71DEFB5
:1010200008F00F9A0F9C0F9E0101000E5E6F600E7C
:101030005F6F3D0E606F080E616F47C100F148C1E0
:1010400001F149C102F14AC103F10101140E046F1B
:10105000050E056F000E066F000E076F61EC1DF0A8
:1010600003AF36EF08F0F2885BEF08F0F2985E6BA2
:101070005F6B606B616B966B976B986B996B9A6B00
:101080009B6B9C6B9D6B9E6B9F6BA06BA16BA26B14
:10109000A36BA46BA56BA66BA76BA86BA96BAA6BC4
:1010A000AB6BAC6BAD6BAE6BAF6BB06BB16BB26B74
:1010B000B36BB46BB56B0CC100F10DC101F10EC186
:1010C00002F10FC103F110C104F111C105F112C108
:1010D00006F113C107F114C108F115C109F116C1D8
:1010E0000AF117C10BF135C134F17DEC21F01C661A
:1010F0001ED01BAE11D01B9E1C8E17AE07D0136ADC
:10110000040E146E156ACAEC1EF011D0136A146A2C
:10111000156ACAEC1EF00BD01BAC09D01B9C1C8CB2
:10112000010E136E146A156ABEEC20F000D08BB469
:10113000A1EF08F010ACA1EF08F08B84109CA2EF97
:1011400008F08B94C3CF55F1C4CF56F1C28207B4D7
:101150000CEF09F047C14BF148C14CF149C14DF1C9
:101160004AC14EF15EC162F15FC163F160C164F1D9
:1011700061C165F196C1B6F197C1B7F198C1B8F1F7
:1011800099C1B9F19AC1BAF19BC1BBF19CC1BCF143
:101190009DC1BDF19EC1BEF19FC1BFF1A0C1C0F113
:1011A000A1C1C1F1A2C1C2F1A3C1C3F1A4C1C4F1E3
:1011B000A5C1C5F1A6C1C6F1A7C1C7F1A8C1C8F1B3
:1011C000A9C1C9F1AAC1CAF1ABC1CBF1ACC1CCF183
:1011D000ADC1CDF1AEC1CEF1AFC1CFF1B0C1D0F153
:1011E000B1C1D1F1B2C1D2F1B3C1D3F1B4C1D4F123
:1011F000B5C1D5F1010155515B2756515C23E86A11
:101200005D230E2E0CEF09F05CC157F15DC158F162
:101210005B6B5C6B5D6B078E0EEF09F002C0E0FF4D
:10122000005001C0D8FF1000A6B214EF09F00CC0A6
:10123000A9FF0BC0A8FFA69EA69CA684F29E550EF1
:10124000A76EAA0EA76EA682F28EA694A6B226EF6D
:1012500009F00C2A1200A96EA69EA69CA680A85092
:101260000C2A120004012C0E826F2BEC0BF05CECAC
:101270001EF00C502BEC09F0E8CF00F10C502BECD9
:1012800009F0E8CF01F101AF4BEF09F00101FF0ECA
:10129000026FFF0E036FFFEC1DF0296757EF09F097
:1012A0000401200E826F2BEC0BF05CEF09F00401BF
:1012B0002D0E826F2BEC0BF029EC1CF01200076A4C
:1012C0000F6A106A116A126A0F010E0EC16E860E45
:1012D000C06E030EC26E0F01896A110E926E080E67
:1012E0008A6EF10E936E8B6A980E946EF18EFC0EE0
:1012F0002BEC09F0E8CF0BF00BA011800BA21182B0
:101300000BA411840BA81188C90E2BEC09F0E8CFAF
:1013100016F0CA0E2BEC09F0E8CF17F0CB0E2BEC31
:1013200009F0E8CF18F0CC0E2BEC09F0E8CF19F05B
:101330001B6A1C6A0E6A01015B6B5C6B5D6B576B11
:10134000586BF29A0101476B486B496B4A6B4B6BC8
:101350004C6B4D6B4E6B4F6B506B516B526B456BC7
:10136000466BD76AD66A0F01280ED56EF28A9D9019
:10137000B00ECD6E01015E6B5F6B606B616B626B7B
:10138000636B646B656B666B676B686B696B536BE8
:10139000546BCF6ACE6A0F9A0F9C0F9E9D80760E7B
:1013A000CA6E9D8202013C0E006FCC6A160E2BECB9
:1013B00009F0E8CF00F1170E2BEC09F0E8CF01F1AE
:1013C000180E2BEC09F0E8CF02F1190E2BEC09F006
:1013D000E8CF03F1010103AF08EF0AF05CEC1EF067
:1013E000160E0C6E00C10BF014EC09F0170E0C6E0B
:1013F00001C10BF014EC09F0180E0C6E02C10BF0D9
:1014000014EC09F0190E0C6E03C10BF014EC09F08A
:1014100000C18AF101C18BF102C18CF103C18DF1D0
:1014200000C18EF101C18FF102C190F103C191F1B0
:101430001A0E2BEC09F0E8CF00F11B0E2BEC09F093
:10144000E8CF01F11C0E2BEC09F0E8CF02F11D0EE4
:101450002BEC09F0E8CF03F1010103AF5EEF0AF0D6
:101460005CEC1EF01A0E0C6E00C10BF014EC09F0CF
:101470001B0E0C6E01C10BF014EC09F01C0E0C6E6F
:1014800002C10BF014EC09F01D0E0C6E03C10BF041
:1014900014EC09F01A0E2BEC09F0E8CF00F11B0E4A
:1014A0002BEC09F0E8CF01F11C0E2BEC09F0E8CF92
:1014B00002F11D0E2BEC09F0E8CF03F100C192F10F
:1014C00001C193F102C194F103C195F1240EAC6EF8
:1014D000900EAB6E240EAC6E080EB86E000EB06EA1
:1014E0001F0EAF6E0401806B816B0F01900EAB6E0F
:1014F0000F019D8A0301806B816BC26B8B92136A13
:10150000146A156A9D8607900001F28EF28C07B06E
:10151000D6EF1AF00FB083EF14F010BE83EF14F083
:1015200012B883EF14F00301805181197F0BD8B4F6
:10153000D6EF1AF013EE00F081517F0BE126812BDC
:10154000E7CFE8FFE00BD8B4D6EF1AF023EE82F035
:10155000C2513F0BD926E7CFDFFFC22BDF50780AFD
:10156000D8A4D6EF1AF007808EC100F18FC101F127
:1015700090C102F191C103F10101040E046F000E4C
:10158000056F000E066F000E076F61EC1DF000AFD7
:10159000D3EF0AF00101030E8E6F000E8F6F000E65
:1015A000906F000E916F03018251720AD8B46EEFF2
:1015B00014F08251520AD8B46EEF14F08251750AB9
:1015C000D8B46EEF14F08251630AD8B490EF17F0DC
:1015D0008251690AD8B41AEF11F082517A0AD8B44C
:1015E0002DEF12F08251490AD8B4B9EF10F08251B0
:1015F000500AD8B4CBEF0FF08251700AD8B411EF73
:1016000010F08251540AD8B43FEF10F08251740A9E
:10161000D8B488EF10F08251410AD8B43FEF0BF0F4
:1016200082516D0AD8B423EF0FF082514D0AD8B41D
:101630003CEF0FF08251730AD8B49EEF13F0825141
:10164000530AD8B403EF14F08251590AD8B474EF96
:101650000EF0C7EF17F0040114EE00F080517F0B7D
:10166000E12682C4E7FF802B120004010D0E826F79
:101670002BEC0BF00A0E826F2BEC0BF01200040126
:10168000410E826F2BEC0BF003018351310AD8B469
:1016900094EF0DF003018351320AD8B4EAEF0CF055
:1016A00003018351330AD8B473EF0CF00301835163
:1016B000340AD8B463EF0BF004013F0E826F2BECB9
:1016C0000BF0C5EF17F0CC0E2BEC09F0E8CF0BF0C8
:1016D00004012C0E826F2BEC0BF003018451310AB4
:1016E000D8B487EF0BF003018451300AD8B489EFE6
:1016F0000BF0030184514D0AD8B493EF0BF00301B2
:101700008451540AD8B49AEF0BF0B1EF0BF08A84ED
:1017100001D08A940BAE04D00BAC02D00BBA21D00E
:10172000E00E0B1218D01F0E0B168539E844E00BA3
:101730000B1211D0E00E0B169DEC1EF085C332F19A
:1017400086C333F10101296BAAEC1EF021EC1EF0D7
:1017500000511F0B0B12CC0E0C6E0BC00BF014ECD7
:1017600009F00401340E826F2BEC0BF004012C0EF7
:10177000826F2BEC0BF0CC0E2BEC09F0E8CF19F0BC
:101780008AB406D00401300E826F2BEC0BF005D02A
:101790000401310E826F2BEC0BF004012C0E826FD2
:1017A0002BEC0BF01938E840070BE8CF82F404016A
:1017B000300E82272BEC0BF004012C0E826F2BECE9
:1017C0000BF05CEC1EF019501F0BE8CF00F1FFECA2
:1017D0001DF032C182F40401300E82272BEC0BF095
:1017E00033C182F40401300E82272BEC0BF004018C
:1017F0002C0E826F2BEC0BF05CEC1EF02CC000F179
:1018000000AF0BD0FF0E016FFF0E026FFF0E036FD4
:1018100004012D0E826F2BEC0BF0FFEC1DF031C19B
:1018200082F40401300E82272BEC0BF032C182F4DB
:101830000401300E82272BEC0BF033C182F404013B
:10184000300E82272BEC0BF004012C0E826F2BEC58
:101850000BF05CEC1EF02BC000F1FFEC1DF031C171
:1018600082F40401300E82272BEC0BF032C182F49B
:101870000401300E82272BEC0BF033C182F40401FB
:10188000300E82272BEC0BF004012C0E826F2BEC18
:101890000BF05CEC1EF02DC000F100AF0BD0FF0E82
:1018A000016FFF0E026FFF0E036F04012D0E826F9A
:1018B0002BEC0BF0FFEC1DF031C182F40401300E73
:1018C00082272BEC0BF032C182F40401300E822708
:1018D0002BEC0BF033C182F40401300E82272BEC89
:1018E0000BF0C5EF17F0CB0E2BEC09F0E8CF0BF0A7
:1018F00004012C0E826F2BEC0BF003018451450A7E
:10190000D8B497EF0CF003018451440AD8B49AEF8D
:101910000CF003018451300AD8B49DEF0CF00301A0
:101920008451310AD8B4A1EF0CF0ACEF0CF00B9E4F
:10193000A6EF0CF00B8EA6EF0CF0FC0E0B16A6EF2C
:101940000CF0FC0E0B160B80A6EF0CF0CB0E0C6E01
:101950000BC00BF014EC09F00401330E826F2BEC7A
:101960000BF004012C0E826F2BEC0BF0CB0E2BEC4A
:1019700009F0E8CF18F018BEC5EF0CF00401450ED1
:10198000826F2BEC0BF0CAEF0CF00401440E826F57
:101990002BEC0BF004012C0E826F2BEC0BF00401EE
:1019A000300E826F2BEC0BF004012C0E826F2BECAF
:1019B0000BF018B0E3EF0CF00401300E826F2BEC4B
:1019C0000BF0E8EF0CF00401310E826F2BEC0BF002
:1019D000C5EF17F0CA0E2BEC09F0E8CF0BF00401AD
:1019E0002C0E826F2BEC0BF003018451450AD8B406
:1019F0001AEF0DF003018451440AD8B41DEF0DF025
:101A0000030184514D0AD8B426EF0DF0030184512F
:101A1000410AD8B420EF0DF003018451460AD8B42E
:101A200023EF0DF003018451560AD8B42EEF0DF0C8
:101A30003FEF0DF00B9E39EF0DF00B8E39EF0DF0EF
:101A40000B9C39EF0DF00B8C39EF0DF0F80E0B16E7
:101A500085C3E8FF070B0B1239EF0DF0C70E0B160D
:101A600085C3E8FF070BE846E846E8460B1239EF66
:101A70000DF0CA0E0C6E0BC00BF014EC09F0CA0E80
:101A80002BEC09F0E8CF17F00401320E826F2BEC3B
:101A90000BF004012C0E826F2BEC0BF017BE58EFED
:101AA0000DF00401450E826F2BEC0BF05DEF0DF095
:101AB0000401440E826F2BEC0BF004012C0E826F9C
:101AC0002BEC0BF017C0E8FF070BE8CF82F4040102
:101AD000300E82272BEC0BF004012C0E826F2BECC6
:101AE0000BF017BC7BEF0DF00401410E826F2BEC65
:101AF0000BF080EF0DF00401460E826F2BEC0BF023
:101B000004012C0E826F2BEC0BF017C0E8FF380B92
:101B1000E842E842E842E8CF82F40401300E82272E
:101B20002BEC0BF0C5EF17F0C90E2BEC09F0E8CF4A
:101B30000BF004012C0E826F2BEC0BF0030184518F
:101B4000450AD8B4B2EF0DF003018451440AD8B469
:101B5000B5EF0DF0030184514D0AD8B4B8EF0DF084
:101B6000C6EF0DF00B9EC0EF0DF00B8EC0EF0DF029
:101B7000F80E0B1685C3E8FF070B0B12C0EF0DF034
:101B8000C90E0C6E0BC00BF014EC09F00401310E01
:101B9000826F2BEC0BF004012C0E826F2BEC0BF000
:101BA000C90E2BEC09F0E8CF16F016BE06D00401E2
:101BB000450E826F2BEC0BF005D00401440E826FB2
:101BC0002BEC0BF004012C0E826F2BEC0BF016C0EB
:101BD000E8FF070BE8CF82F40401300E82272BECDC
:101BE0000BF004012C0E826F2BEC0BF007805CECE9
:101BF0001EF027C0E8FF003B00430043030BFFEC4F
:101C00001DF033C182F40401300E82272BEC0BF05F
:101C100004012C0E826F2BEC0BF05CEC1EF027C045
:101C200001F1019F019D28C000F10101FFEC1DF0B1
:101C30002FC182F40401300E82272BEC0BF030C14F
:101C400082F40401300E82272BEC0BF031C182F4B8
:101C50000401300E82272BEC0BF032C182F4040118
:101C6000300E82272BEC0BF033C182F40401300ECE
:101C700082272BEC0BF004012C0E826F2BEC0BF067
:101C80005CEC1EF029C001F12AC000F1D8900133AC
:101C90000033D890013300330101FFEC1DF02FC158
:101CA00082F40401300E82272BEC0BF030C182F459
:101CB0000401300E82272BEC0BF031C182F40401B9
:101CC000300E82272BEC0BF032C182F40401300E6F
:101CD00082272BEC0BF033C182F40401300E8227F3
:101CE0002BEC0BF0C5EF17F0FC0E2BEC09F0E8CF56
:101CF0000BF003018351520AD8B4ABEF0EF003018D
:101D00008351720AD8B4AEEF0EF003018351500A2A
:101D1000D8B4B1EF0EF003018351700AD8B4B4EF18
:101D20000EF003018351550AD8B4B7EF0EF003014A
:101D30008351750AD8B4BAEF0EF003018351430AF8
:101D4000D8B4C3EF0EF003018351630AD8B4C6EFD1
:101D50000EF0CFEF0EF00B90C9EF0EF00B80C9EF35
:101D60000EF00B92C9EF0EF00B82C9EF0EF00B9440
:101D7000C9EF0EF00B84C9EF0EF00B96C9EF0EF011
:101D80000B86C9EF0EF00B98C9EF0EF00B88C9EF68
:101D90000EF0FC0E0C6E0BC00BF014EC09F00401FD
:101DA000590E826F2BEC0BF0119011921194119837
:101DB000FC0E2BEC09F0E8CF0BF00BA011800BA26E
:101DC00011820BA411840BA8118811A0EFEF0EF063
:101DD0000401520E826F2BEC0BF0F4EF0EF00401B5
:101DE000720E826F2BEC0BF011A8FEEF0EF00401C7
:101DF000430E826F2BEC0BF003EF0FF00401630E28
:101E0000826F2BEC0BF011A20DEF0FF00401500EBE
:101E1000826F2BEC0BF012EF0FF00401700E826F4B
:101E20002BEC0BF011A41CEF0FF00401550E826F88
:101E30002BEC0BF021EF0FF00401750E826F2BECF1
:101E40000BF0C5EF17F004016D0E826F2BEC0BF059
:101E500003018351300AD8B47BEF0FF003018351A3
:101E6000310AD8B48EEF0FF003018351320AD8B48F
:101E7000A1EF0FF0C7EF17F004014D0E826F2BECAE
:101E80000BF09DEC1EF084C331F185C332F186C3A3
:101E900033F10101296BAAEC1EF021EC1EF00301C5
:101EA0008351300AD8B463EF0FF003018351310A34
:101EB000D8B46BEF0FF003018351320AD8B473EF3B
:101EC0000FF0C7EF17F0FD0E0C6E00C10BF014EC15
:101ED00009F07BEF0FF0FE0E0C6E00C10BF014EC5E
:101EE00009F08EEF0FF0FF0E0C6E00C10BF014EC3A
:101EF00009F0A1EF0FF00401300E826F2BEC0BF014
:101F000004012C0E826F2BEC0BF05CEC1EF0FD0E2E
:101F10002BEC09F0E8CF00F1B2EF0FF00401310E25
:101F2000826F2BEC0BF004012C0E826F2BEC0BF06C
:101F30005CEC1EF0FE0E2BEC09F0E8CF00F1B2EFE6
:101F40000FF00401320E826F2BEC0BF05CEC1EF0F4
:101F500004012C0E826F2BEC0BF0FF0E2BEC09F022
:101F6000E8CF00F1FFEC1DF031C182F40401300E26
:101F700082272BEC0BF032C182F40401300E822751
:101F80002BEC0BF033C182F40401300E82272BECD2
:101F90000BF0C5EF17F081A8B9EF10F083C32AF159
:101FA00084C32BF185C32CF186C32DF187C32EF199
:101FB00088C32FF189C330F18AC331F18BC332F169
:101FC0008CC333F10101AAEC1EF021EC1EF0160EB9
:101FD0000C6E00C10BF014EC09F0170E0C6E01C171
:101FE0000BF014EC09F0180E0C6E02C10BF014EC9F
:101FF00009F0190E0C6E03C10BF014EC09F000C1CE
:102000008AF101C18BF102C18CF103C18DF100C1D4
:102010008EF101C18FF102C190F103C191F1B9EFCD
:1020200010F081A8B9EF10F083C32AF184C32BF11B
:1020300085C32CF186C32DF187C32EF188C32FF100
:1020400089C330F18AC331F18BC332F18CC333F1D0
:102050000101AAEC1EF021EC1EF000C18AF101C1C1
:102060008BF102C18CF103C18DF100C18EF101C170
:102070008FF102C190F103C191F1B9EF10F081A885
:10208000B9EF10F083C32AF184C32BF185C32CF17F
:1020900086C32DF187C32EF188C32FF189C330F198
:1020A0008AC331F18CC332F18DC333F10101AAEC43
:1020B0001EF021EC1EF00101000E046F000E056FF2
:1020C000010E066F000E076F72EC1DF01A0E0C6EFB
:1020D00000C10BF014EC09F01B0E0C6E01C10BF0EB
:1020E00014EC09F01C0E0C6E02C10BF014EC09F09C
:1020F0001D0E0C6E03C10BF014EC09F000C192F13F
:1021000001C193F102C194F103C195F1B9EF10F04F
:1021100081A8B9EF10F083C32AF184C32BF185C3E2
:102120002CF186C32DF187C32EF188C32FF189C30B
:1021300030F18AC331F18CC332F18DC333F1010127
:10214000AAEC1EF021EC1EF00101000E046F000E3F
:10215000056F010E066F000E076F72EC1DF000C1D7
:1021600092F101C193F102C194F103C195F1B9EF6C
:1021700010F0160E2BEC09F0E8CF00F1170E2BEC47
:1021800009F0E8CF01F1180E2BEC09F0E8CF02F1CD
:10219000190E2BEC09F0E8CF03F1FFEC1DF0E2EC97
:1021A0001BF00401730E826F2BEC0BF004012C0E5C
:1021B000826F2BEC0BF08AC100F18BC101F18CC155
:1021C00002F18DC103F1FFEC1DF0E2EC1BF0040104
:1021D000730E826F2BEC0BF004012C0E826F2BEC34
:1021E0000BF01A0E2BEC09F0E8CF00F11B0E2BECD4
:1021F00009F0E8CF01F11C0E2BEC09F0E8CF02F159
:102200001D0E2BEC09F0E8CF03F1E2EC17F004010E
:102210002C0E826F2BEC0BF092C100F193C101F1F7
:1022200094C102F195C103F1E2EC17F035EC0BF02B
:10223000C7EF17F00401690E826F2BEC0BF004015D
:102240002C0E826F2BEC0BF00101040E006F000EC0
:10225000016F000E026F000E036FFFEC1DF02CC12A
:1022600082F40401300E82272BEC0BF02DC182F496
:102270000401300E82272BEC0BF02EC182F40401F6
:10228000300E82272BEC0BF02FC182F40401300EAC
:1022900082272BEC0BF030C182F40401300E822730
:1022A0002BEC0BF031C182F40401300E82272BECB1
:1022B0000BF032C182F40401300E82272BEC0BF0BC
:1022C00033C182F40401300E82272BEC0BF00401A1
:1022D0002C0E826F2BEC0BF00101030E006F000E31
:1022E000016F000E026F000E036FFFEC1DF02CC19A
:1022F00082F40401300E82272BEC0BF02DC182F406
:102300000401300E82272BEC0BF02EC182F4040165
:10231000300E82272BEC0BF02FC182F40401300E1B
:1023200082272BEC0BF030C182F40401300E82279F
:102330002BEC0BF031C182F40401300E82272BEC20
:102340000BF032C182F40401300E82272BEC0BF02B
:1023500033C182F40401300E82272BEC0BF0040110
:102360002C0E826F2BEC0BF001012B0E006F000E78
:10237000016F000E026F000E036FFFEC1DF02CC109
:1023800082F40401300E82272BEC0BF02DC182F475
:102390000401300E82272BEC0BF02EC182F40401D5
:1023A000300E82272BEC0BF02FC182F40401300E8B
:1023B00082272BEC0BF030C182F40401300E82270F
:1023C0002BEC0BF031C182F40401300E82272BEC90
:1023D0000BF032C182F40401300E82272BEC0BF09B
:1023E00033C182F40401300E82272BEC0BF0040180
:1023F0002C0E826F2BEC0BF0200EF86EF76AF66A4B
:1024000004010900F5CF82F42BEC0BF00900F5CFA5
:1024100082F42BEC0BF00900F5CF82F42BEC0BF0DF
:102420000900F5CF82F42BEC0BF00900F5CF82F414
:102430002BEC0BF00900F5CF82F42BEC0BF009002C
:10244000F5CF82F42BEC0BF00900F5CF82F42BECE6
:102450000BF035EC0BF0C7EF17F08351630AD8A4EB
:10246000C7EF17F08451610AD8A4C7EF17F0855160
:102470006C0AD8A4C7EF17F08651410A42E0865192
:10248000440A1BE08651420AD8B494EF12F08651F8
:10249000350AD8B451EF19F08651360AD8B4A6EFF0
:1024A00019F08651370AD8B40FEF1AF08651380A5E
:1024B000D8B46DEF1AF0C7EF17F00798079A040128
:1024C0007A0E826F2BEC0BF00401780E826F2BECEE
:1024D0000BF00401640E826F2BEC0BF081A878EFF7
:1024E00012F00401550E826F2BEC0BF07DEF12F011
:1024F00004014C0E826F2BEC0BF035EC0BF0C7EFA8
:1025000017F00788079A04017A0E826F2BEC0BF004
:102510000401410E826F2BEC0BF00401610E826FFF
:102520002BEC0BF06EEF12F00798078A04017A0E7D
:10253000826F2BEC0BF00401420E826F2BEC0BF040
:102540000401610E826F2BEC0BF06EEF12F00101B3
:102550006667B2EF12F06767B2EF12F06867B2EF2A
:1025600012F0696715D04F67BDEF12F05067BDEFED
:1025700012F05167BDEF12F052670AD00101000E50
:10258000006F000E016F000E026F000E036F12004D
:1025900011B80AD00101620E046F010E056F000E22
:1025A000066F000E076F09D00101A70E046F020E1F
:1025B000056F000E066F000E076F66C100F167C160
:1025C00001F168C102F169C103F161EC1DF003BFC3
:1025D0005AEF13F0119A119C0101000E046FA80E1E
:1025E000056F550E066F020E076F66C100F167C1D9
:1025F00001F168C102F169C103F166C186F167C1E9
:1026000087F168C188F169C189F161EC1DF003BFF0
:102610000BD00101000E866FA80E876F550E886FD4
:10262000020E896F118A119C0E0E2BEC09F0E8CF77
:1026300018F10F0E2BEC09F0E8CF19F1100E2BEC6E
:1026400009F0E8CF1AF1110E2BEC09F0E8CF1BF1DD
:10265000AAEC1CF086C104F187C105F188C106F11E
:1026600089C107F161EC1DF007826EEC1CF0AAEC49
:102670001CF007926EEC1CF086C100F187C101F1DD
:1026800088C102F189C103F107926EEC1CF0CC0EF7
:10269000046FE00E056F870E066F050E076F61EC85
:1026A0001DF000C118F101C119F102C11AF103C1F5
:1026B0001BF13BD0119C119A0101800E006F1A0E84
:1026C000016F060E026F000E036F4FC104F150C17F
:1026D00005F151C106F152C107F161EC1DF003AFE4
:1026E00005D05CEC1EF0118C119A12000E0E2BEC32
:1026F00009F0E8CF18F10F0E2BEC09F0E8CF19F133
:10270000100E2BEC09F0E8CF1AF1110E2BEC09F0AA
:10271000E8CF1BF14FC100F150C101F151C102F1ED
:1027200052C103F107826EEC1CF018C100F119C10F
:1027300001F11AC102F11BC103F112000401730E71
:10274000826F2BEC0BF004012C0E826F2BEC0BF044
:10275000078462C166F163C167F164C168F165C154
:1027600069F14BC14FF14CC150F14DC151F14EC116
:1027700052F157C159F158C15AF10794C4EC13F002
:1027800035EC0BF0C7EF17F066C100F167C101F13E
:1027900068C102F169C103F10101FFEC1DF0E2EC37
:1027A0001BF00401630E826F2BEC0BF004012C0E66
:1027B000826F2BEC0BF04FC100F150C101F151C100
:1027C00002F152C103F10101FFEC1DF0E2EC1BF03C
:1027D0000401660E826F2BEC0BF004012C0E826F4D
:1027E0002BEC0BF05CEC1EF059C100F15AC101F169
:1027F0000101FFEC1DF0E2EC1BF00401740E826F8E
:102800002BEC0BF0120010820401530E826F2BECA4
:102810000BF004012C0E826F2BEC0BF083C32AF11A
:1028200084C32BF185C32CF186C32DF187C32EF110
:1028300088C32FF189C330F18AC331F18BC332F1E0
:102840008CC333F10101AAEC1EF021EC1EF000C193
:1028500066F101C167F102C168F103C169F18EC37C
:102860002AF18FC32BF190C32CF191C32DF192C3A8
:102870002EF193C32FF194C330F195C331F196C378
:1028800032F197C333F10101AAEC1EF021EC1EF0E6
:1028900000C14FF101C150F102C151F103C152F128
:1028A0009DEC1EF099C32FF19AC330F19BC331F117
:1028B0009CC332F19DC333F10101AAEC1EF021EC5F
:1028C0001EF000C159F101C15AF1C4EC13F004012A
:1028D0002C0E826F2BEC0BF077EF14F018A001D0C8
:1028E000108C8251520A02E10F8201D00F92825164
:1028F000750A02E1108401D010948251550A02E158
:10290000108601D0109611A003D011A401D010841C
:10291000078410B2E5EF14F010A4D1EF14F0B6C1A3
:1029200066F1B7C167F1B8C168F1B9C169F1BAC15F
:102930006AF1BBC16BF1BCC16CF1BDC16DF1BEC12F
:102940006EF1BFC16FF1C0C170F1C1C171F1C2C1FF
:1029500072F1C3C173F1C4C174F1C5C175F1C6C1CF
:1029600076F1C7C177F1C8C178F1C9C179F1CAC19F
:102970007AF1CBC17BF1CCC17CF1CDC17DF1CEC16F
:102980007EF1CFC17FF1D0C180F1D1C181F1D2C13F
:1029900082F1D3C183F1D4C184F1D5C185F1D9EFDE
:1029A00014F062C166F163C167F164C168F165C189
:1029B00069F14BC14FF14CC150F14DC151F14EC1C4
:1029C00052F157C159F158C15AF107940FA007EFBE
:1029D00015F001019267F4EF14F09367F4EF14F02F
:1029E0009467F4EF14F09567F8EF14F007EF15F023
:1029F000A7EC12F092C104F193C105F194C106F164
:102A000095C107F161EC1DF003BF8DEF17F0A7EC46
:102A100012F00101000E046F000E056F010E066F2B
:102A2000000E076F92EC1DF011A02CD011A22AD03D
:102A3000FFEC1DF0296701D007D004012D0E826F35
:102A40002BEC0BF08BEF17F030C182F40401300E49
:102A500082272BEC0BF031C182F40401300E822767
:102A60002BEC0BF032C182F40401300E82272BECE8
:102A70000BF033C182F40401300E82272BEC0BF0F3
:102A80008BEF17F012A8C5D0129819C01AF01A3A95
:102A90001A42070E1A1600011A50000AD8B4D5EFD0
:102AA00015F000011A50010AD8B461EF15F00001C9
:102AB0001A50020AD8B45FEF15F007EF16F007EFCF
:102AC00016F05CEC1EF029C001F12AC000F1D8908C
:102AD00001330033D890013300330101630E046FDA
:102AE000000E056F000E066F000E076F92EC1DF0D2
:102AF000280E046F000E056F000E066F000E076FA4
:102B000061EC1DF000C12CF05CEC1EF027C001F15F
:102B1000019F019D28C000F10101A40E046F000E69
:102B2000056F000E066F000E076F92EC1DF000C1DE
:102B30002BF000C104F101C105F102C106F103C18E
:102B400007F1640E006F000E016F000E026F000EA1
:102B5000036F61EC1DF0050E046F000E056F000E93
:102B6000066F000E076F92EC1DF000C104F101C169
:102B700005F102C106F103C107F15CEC1EF02CC0A7
:102B800000F161EC1DF000C12DF02DC0E8FF050F34
:102B90002C5C03E78A8407EF16F02DC0E8FF0A0FCC
:102BA0002C5C01E68A9407EF16F000C124F101C104
:102BB00025F102C126F103C127F15CEC1EF062ECA5
:102BC0001EF019501F0BE8CF00F10101640E046FD5
:102BD000000E056F000E066F000E076F72EC1DF001
:102BE00024C104F125C105F126C106F127C107F171
:102BF00061EC1DF003BF02D08A9401D08A8424C105
:102C000000F125C101F126C102F127C103F18DEFC9
:102C100017F010AE4BD0109E00C108F101C109F1B0
:102C200002C10AF103C10BF1FFEC1DF030C1D6F176
:102C300031C1D7F132C1D8F133C1D9F108C100F1A6
:102C400009C101F10AC102F10BC103F101016C0ECE
:102C5000046F070E056F000E066F000E076F61EC24
:102C60001DF003BF04D00101550EDA6F1CD008C15E
:102C700000F109C101F10AC102F10BC103F1010127
:102C8000A40E046F060E056F000E066F000E076F90
:102C900061EC1DF003BF04D001017F0EDA6F03D099
:102CA0000101FF0EDA6F1B8E8DEF17F010A460EF9D
:102CB00016F00401750E826F2BEC0BF065EF16F029
:102CC0000401720E826F2BEC0BF004012C0E826F4C
:102CD0002BEC0BF0FFEC1DF0296774EF16F00401EC
:102CE000200E826F77EF16F004012D0E826F2BEC11
:102CF0000BF030C182F40401300E82272BEC0BF074
:102D000031C182F40401300E82272BEC0BF0040158
:102D10002E0E826F2BEC0BF032C182F40401300EC8
:102D200082272BEC0BF033C182F40401300E822792
:102D30002BEC0BF004016D0E826F2BEC0BF00401F9
:102D40002C0E826F2BEC0BF04FC100F150C101F142
:102D500051C102F152C103F10101FFEC1DF0E2EC9F
:102D60001BF00401480E826F2BEC0BF004017A0E6D
:102D7000826F2BEC0BF004012C0E826F2BEC0BF00E
:102D800066C100F167C101F168C102F169C103F1D7
:102D90000101FFEC1DF0E2EC1BF00401630E826FF9
:102DA0002BEC0BF004012C0E826F2BEC0BF066C1A8
:102DB00000F167C101F168C102F169C103F10101CC
:102DC0000A0E046F000E056F000E066F000E076FEF
:102DD00072EC1DF0000E046F120E056F000E066FF0
:102DE000000E076F92EC1DF0FFEC1DF02AC182F47B
:102DF0000401300E82272BEC0BF02BC182F404016E
:102E0000300E82272BEC0BF02CC182F40401300E23
:102E100082272BEC0BF02DC182F40401300E8227A7
:102E20002BEC0BF02EC182F40401300E82272BEC28
:102E30000BF02FC182F40401300E82272BEC0BF033
:102E400030C182F40401300E82272BEC0BF0040118
:102E50002E0E826F2BEC0BF031C182F40401300E88
:102E600082272BEC0BF032C182F40401300E822752
:102E70002BEC0BF033C182F40401300E82272BECD3
:102E80000BF00401730E826F2BEC0BF004012C0E7F
:102E9000826F2BEC0BF05CEC1EF059C100F15AC1B3
:102EA00001F1F1EC18F00FB259EF17F00FA08BEF12
:102EB00017F004012C0E826F2BEC0BF0200EF86E35
:102EC000F76AF66A04010900F5CF82F42BEC0BF0E7
:102ED0000900F5CF82F42BEC0BF00900F5CF82F45A
:102EE0002BEC0BF00900F5CF82F42BEC0BF0090072
:102EF000F5CF82F42BEC0BF00900F5CF82F42BEC2C
:102F00000BF00900F5CF82F42BEC0BF00900F5CFA4
:102F100082F42BEC0BF035EC0BF00F90C7EF17F0B1
:102F20000401630E826F2BEC0BF004012C0E826FF8
:102F30002BEC0BF0CDEC17F004012C0E826F2BEC78
:102F40000BF040EC18F004012C0E826F2BEC0BF010
:102F5000BCEC18F004012C0E826F2BEC0BF001017D
:102F6000F80E006FCD0E016F660E026F030E036F39
:102F7000E2EC17F004012C0E826F2BEC0BF0D2EC7C
:102F800018F035EC0BF0C7EF17F035EC0BF0030140
:102F9000C26B07901092D6EF1AF0D8900E0E2BEC61
:102FA00009F0E8CF00F10F0E2BEC09F0E8CF01F1AA
:102FB000100E2BEC09F0E8CF02F1110E2BEC09F00A
:102FC000E8CF03F10101000E046F000E056F010E42
:102FD000066F000E076F92EC1DF0FFEC1DF02AC18A
:102FE00082F40401300E82272BEC0BF02BC182F40B
:102FF0000401300E82272BEC0BF02CC182F404016B
:10300000300E82272BEC0BF02DC182F40401300E20
:1030100082272BEC0BF02EC182F40401300E8227A4
:103020002BEC0BF02FC182F40401300E82272BEC25
:103030000BF030C182F40401300E82272BEC0BF030
:1030400031C182F40401300E82272BEC0BF0040115
:103050002E0E826F2BEC0BF032C182F40401300E85
:1030600082272BEC0BF033C182F40401300E82274F
:103070002BEC0BF004016D0E826F2BEC0BF01200A9
:10308000120E2BEC09F0E8CF00F1130E2BEC09F037
:10309000E8CF01F1140E2BEC09F0E8CF02F1150E88
:1030A0002BEC09F0E8CF03F101010A0E046F000ECA
:1030B000056F000E066F000E076F72EC1DF0000E1C
:1030C000046F120E056F000E066F000E076F92EC74
:1030D0001DF0FFEC1DF02AC182F40401300E82279E
:1030E0002BEC0BF02BC182F40401300E82272BEC69
:1030F0000BF02CC182F40401300E82272BEC0BF074
:103100002DC182F40401300E82272BEC0BF02EC16E
:1031100082F40401300E82272BEC0BF02FC182F4D5
:103120000401300E82272BEC0BF030C182F4040135
:10313000300E82272BEC0BF004012E0E826F2BEC4D
:103140000BF031C182F40401300E82272BEC0BF01E
:1031500032C182F40401300E82272BEC0BF033C114
:1031600082F40401300E82272BEC0BF00401730E65
:10317000826F2BEC0BF012000A0E2BEC09F0E8CF5B
:1031800000F10B0E2BEC09F0E8CF01F10C0E2BEC4B
:1031900009F0E8CF02F10D0E2BEC09F0E8CF03F1B6
:1031A000F1EF18F0060E2BEC09F0E8CF00F1070E56
:1031B0002BEC09F0E8CF01F1080E2BEC09F0E8CF79
:1031C00002F1090E2BEC09F0E8CF03F1F1EF18F052
:1031D00001015CEC1EF0078457C100F158C101F1F8
:1031E00007940101E80E046F800E056F000E066F54
:1031F000000E076F72EC1DF0000E046F040E056FD9
:10320000000E066F000E076F92EC1DF0880E046F23
:10321000130E056F000E066F000E076F61EC1DF0B8
:103220000A0E046F000E056F000E066F000E076F8A
:1032300092EC1DF0FFEC1DF00101296725EF19F05C
:103240000401200E826F28EF19F004012D0E826F09
:103250002BEC0BF030C182F40401300E82272BECF2
:103260000BF031C182F40401300E82272BEC0BF0FD
:1032700032C182F40401300E82272BEC0BF00401E2
:103280002E0E826F2BEC0BF033C182F40401300E52
:1032900082272BEC0BF00401430E826F2BEC0BF01A
:1032A000120087C32AF188C32BF189C32CF18AC38A
:1032B0002DF18BC32EF18CC32FF18DC330F18EC352
:1032C00031F190C332F191C333F10101296BAAECC2
:1032D0001EF021EC1EF00101000E046F000E056FC0
:1032E000010E066F000E076F72EC1DF00E0E0C6ED5
:1032F00000C10BF014EC09F00F0E0C6E01C10BF0C5
:1033000014EC09F0100E0C6E02C10BF014EC09F075
:10331000110E0C6E03C10BF014EC09F004017A0ECF
:10332000826F2BEC0BF004012C0E826F2BEC0BF058
:103330000401350E826F2BEC0BF004012C0E826F12
:103340002BEC0BF0CDEC17F07DEF12F087C32AF1D8
:1033500088C32BF189C32CF18AC32DF18BC32EF1C5
:103360008CC32FF18DC330F18EC331F190C332F194
:1033700091C333F10101296BAAEC1EF021EC1EF080
:10338000880E046F130E056F000E066F000E076F98
:1033900066EC1DF0000E046F040E056F000E066F44
:1033A000000E076F72EC1DF00101E80E046F800E35
:1033B000056F000E066F000E076F92EC1DF00A0EEF
:1033C0000C6E00C10BF014EC09F00B0E0C6E01C179
:1033D0000BF014EC09F00C0E0C6E02C10BF014ECA7
:1033E00009F00D0E0C6E03C10BF014EC09F0040192
:1033F0007A0E826F2BEC0BF004012C0E826F2BECFB
:103400000BF00401360E826F2BEC0BF004012C0E36
:10341000826F2BEC0BF0BCEC18F07DEF12F087C341
:103420002AF188C32BF189C32CF18AC32DF18BC3F8
:103430002EF18CC32FF18DC330F18FC331F190C3C6
:1034400032F191C333F10101AAEC1EF021EC1EF020
:10345000000E046F120E056F000E066F000E076F50
:1034600072EC1DF001010A0E046F000E056F000ED4
:10347000066F000E076F92EC1DF0120E0C6E00C16D
:103480000BF014EC09F0130E0C6E01C10BF014ECF0
:1034900009F0140E0C6E02C10BF014EC09F0150EBD
:1034A0000C6E03C10BF014EC09F004017A0E826F6C
:1034B0002BEC0BF004012C0E826F2BEC0BF00401B3
:1034C000370E826F2BEC0BF004012C0E826F2BEC6D
:1034D0000BF040EC18F07DEF12F087C32AF188C39F
:1034E0002BF189C32CF18AC32DF18BC32EF18CC330
:1034F0002FF18DC330F18EC331F190C332F191C3FE
:1035000033F10101296BAAEC1EF021EC1EF0880EAC
:10351000046F130E056F000E066F000E076F66EC4A
:103520001DF0000E046F040E056F000E066F000EF6
:10353000076F72EC1DF00101E80E046F800E056F3D
:10354000000E066F000E076F92EC1DF0060E0C6E5B
:1035500000C10BF014EC09F0070E0C6E01C10BF06A
:1035600014EC09F0080E0C6E02C10BF014EC09F01B
:10357000090E0C6E03C10BF014EC09F004017A0E75
:10358000826F2BEC0BF004012C0E826F2BEC0BF0F6
:103590000401380E826F2BEC0BF004012C0E826FAD
:1035A0002BEC0BF0D2EC18F07DEF12F081A894EF29
:1035B0001BF007A84DEF1BF00101800E006F1A0EE3
:1035C000016F060E026F000E036F4BC104F14CC178
:1035D00005F14DC106F14EC107F161EC1DF003BFCD
:1035E00094EF1BF0DCEC1BF04BC100F14CC101F17E
:1035F0004DC102F14EC103F107826EEC1CF018C1FF
:1036000004F119C105F11AC106F11BC107F1F80E49
:10361000006FCD0E016F660E026F030E036F61EC3B
:103620001DF00E0E0C6E00C10BF014EC09F00F0E25
:103630000C6E01C10BF014EC09F0100E0C6E02C1FF
:103640000BF014EC09F0110E0C6E03C10BF014EC2E
:1036500009F0078401015CEC1EF057C100F158C16C
:1036600001F107940A0E0C6E00C10BF014EC09F086
:103670000B0E0C6E01C10BF014EC09F00C0E0C6E6D
:1036800002C10BF014EC09F00D0E0C6E03C10BF02F
:1036900014EC09F0079894EF1BF007AA94EF1BF0C5
:1036A000078401015CEC1EF057C100F158C101F123
:1036B0000794060E0C6E00C10BF014EC09F0070E17
:1036C0000C6E01C10BF014EC09F0080E0C6E02C177
:1036D0000BF014EC09F0090E0C6E03C10BF014ECA6
:1036E00009F0078462C100F163C101F164C102F114
:1036F00065C103F10794120E0C6E00C10BF014ECBF
:1037000009F0130E0C6E01C10BF014EC09F0140E4D
:103710000C6E02C10BF014EC09F0150E0C6E03C117
:103720000BF014EC09F0079A0401805181197F0B0A
:103730000BE09EA809D014EE00F081517F0BE1262A
:10374000E750812B0F01AD6E87EF0AF018C100F131
:1037500019C101F11AC102F11BC103F1000E046F7E
:10376000000E056F010E066F000E076F92EC1DF044
:1037700029A1D1EF1BF02051D8B4D1EF1BF018C113
:1037800000F119C101F11AC102F11BC103F1000ED0
:10379000046F000E056F0A0E066F000E076F92ECA5
:1037A0001DF01200010104510013055101130651CF
:1037B00002130751031312000101186B196B1A6BE6
:1037C0001B6B12002AC182F40401300E82272BECFD
:1037D0000BF02BC182F40401300E82272BEC0BF08E
:1037E0002CC182F40401300E82272BEC0BF02DC18A
:1037F00082F40401300E82272BEC0BF02EC182F4F0
:103800000401300E82272BEC0BF02FC182F404014F
:10381000300E82272BEC0BF030C182F40401300E05
:1038200082272BEC0BF031C182F40401300E822789
:103830002BEC0BF032C182F40401300E82272BEC0A
:103840000BF033C182F40401300E82272BEC0BF015
:1038500012002FC182F40401300E82272BEC0BF0F2
:1038600030C182F40401300E82272BEC0BF031C101
:1038700082F40401300E82272BEC0BF032C182F46B
:103880000401300E82272BEC0BF033C182F40401CB
:10389000300E82272BEC0BF01200060E1D6E060E6A
:1038A0001E6E060E1F6E1D2E53EF1CF01E2E53EFC4
:1038B0001CF01F2E53EF1CF08B84020E1D6E020EA7
:1038C0001E6E020E1F6E1D2E63EF1CF01E2E63EF88
:1038D0001CF01F2E63EF1CF08B94120001010053AB
:1038E00005E1015303E1025301E1002B31EC1DF02E
:1038F0005CEC1EF03951006F3A51016F420E046FBB
:103900004B0E056F000E066F000E076F72EC1DF078
:1039100000C104F101C105F102C106F103C107F1C3
:1039200018C100F119C101F11AC102F11BC103F163
:1039300007B29FEF1CF066EC1DF0A1EF1CF061ECEC
:103940001DF000C118F101C119F102C11AF103C142
:103950001BF112005CEC1EF059C100F15AC101F1DB
:10396000060E2BEC09F0E8CF04F1070E2BEC09F062
:10397000E8CF05F1080E2BEC09F0E8CF06F1090EAF
:103980002BEC09F0E8CF07F161EC1DF000C124F148
:1039900001C125F102C126F103C127F1290E046FEF
:1039A000000E056F000E066F000E076F72EC1DF023
:1039B000EE0E046F430E056F000E066F000E076FCC
:1039C00066EC1DF024C104F125C105F126C106F104
:1039D00027C107F172EC1DF000C11CF101C11DF1FE
:1039E00002C11EF103C11FF1120E2BEC09F0E8CF4A
:1039F00004F1130E2BEC09F0E8CF05F1140E2BECBB
:103A000009F0E8CF06F1150E2BEC09F0E8CF07F12D
:103A10000D0E006F000E016F000E026F000E036F9F
:103A200072EC1DF0180E046F000E056F000E066F8D
:103A3000000E076F92EC1DF01CC104F11DC105F1D1
:103A40001EC106F11FC107F166EC1DF06A0E046F7E
:103A50002A0E056F000E066F000E076F61EC1DF059
:103A60001200BF0EFA6E200E3A6F396BD8900037F5
:103A7000013702370337D8B042EF1DF03A2F37EF46
:103A80001DF039073A070353D8B412000331070B6E
:103A900080093F6F03390F0B010F396F80EC5FF026
:103AA000406F390580EC5FF0405D405F396B3F331C
:103AB000D8B0392739333FA957EF1DF04051392786
:103AC0001200010181EC1EF0D8B012000101035177
:103AD0000719346F44EC1EF0D8900751031934AF26
:103AE000800F12000101346B68EC1EF0D8A07EEC50
:103AF0001EF0D8B0120053EC1EF05CEC1EF01F0E4E
:103B0000366F94EC1EF00B35D8B044EC1EF0D8A004
:103B10000335D8B01200362F81EF1DF034B16BECB5
:103B20001EF012000101346B04510511061107113A
:103B30000008D8A068EC1EF0D8A07EEC1EF0D8B02B
:103B40001200086B096B0A6B0B6B94EC1EF01F0ED6
:103B5000366F94EC1EF007510B5DD8A4BCEF1DF03E
:103B600006510A5DD8A4BCEF1DF00551095DD8A42B
:103B7000BCEF1DF00451085DD8A0CFEF1DF004513B
:103B8000085F0551D8A0053D095F0651D8A0063D44
:103B90000A5F0751D8A0073D0B5FD8900081362FF0
:103BA000A9EF1DF034B16BEC1EF0346B68EC1EF025
:103BB000D89098EC1EF007510B5DD8A4ECEF1DF0E7
:103BC00006510A5DD8A4ECEF1DF00551095DD8A49B
:103BD000ECEF1DF00451085DD8A0FBEF1DF0003F95
:103BE000FBEF1DF0013FFBEF1DF0023FFBEF1DF06F
:103BF000032BD8B4120034B16BEC1EF0120001019B
:103C0000346B68EC1EF0D8B012009DEC1EF0200E54
:103C1000366F003701370237033711EE33F00A0EE3
:103C2000376FE7360A0EE75CD8B0E76EE552372FFC
:103C300011EF1EF0362F09EF1EF034B12981D89014
:103C4000120001010A0E346F200E366F11EE29F0BA
:103C50003451376F0A0ED890E652D8B0E726E732D3
:103C6000372F2CEF1EF00333023301330033362F8E
:103C700026EF1EF0E750FF0FD8A00335D8B0120092
:103C800029B16BEC1EF01200045100270551D8B089
:103C9000053D01270651D8B0063D02270751D8B08F
:103CA000073D032712000051086F0151096F0251AF
:103CB0000A6F03510B6F12000101006B016B026B65
:103CC000036B12000101046B056B066B076B12009E
:103CD0000335D8A012000351800B001F011F021FE3
:103CE000031F003F7BEF1EF0013F7BEF1EF0023F02
:103CF0007BEF1EF0032B342B032512000735D8A0D1
:103D000012000751800B041F051F061F071F043FE9
:103D100091EF1EF0053F91EF1EF0063F91EF1EF070
:103D2000072B342B072512000037013702370337E2
:103D3000083709370A370B3712000101296B2A6B44
:103D40002B6B2C6B2D6B2E6B2F6B306B316B326BA7
:103D5000336B120001012A510F0B2A6F2B510F0BED
:103D60002B6F2C510F0B2C6F2D510F0B2D6F2E51D4
:103D70000F0B2E6F2F510F0B2F6F30510F0B306F1A
:103D800031510F0B316F32510F0B326F33510F0B1B
:103D9000336F120000011550FF0A01E11200390EC5
:103DA000C86E800EC76E280EC66E000EC56E14500B
:103DB000000AD8B405EF1FF01450010AD8B41EEF62
:103DC0001FF01450020AD8B437EF1FF01450030A42
:103DD000D8B450EF1FF01450040AD8B478EF1FF095
:103DE0001450050AD8B491EF1FF01450060AD8B445
:103DF000AAEF1FF01450070AD8B4C3EF1FF01450F5
:103E0000080AD8B4DCEF1FF012001550000AD8B42D
:103E1000FBEF1FF01550010AD8B4FFEF1FF015504B
:103E2000020AD8B403EF20F01550030AD8B407EF04
:103E300020F01550040AD8B476EF20F01550000A8F
:103E4000D8B40BEF20F01550010AD8B40FEF20F0D2
:103E50001550020AD8B413EF20F01550030AD8B455
:103E600017EF20F01550040AD8B476EF20F0155063
:103E7000000AD8B41BEF20F01550010AD8B41FEF88
:103E800020F01550020AD8B423EF20F01550030A91
:103E9000D8B427EF20F01550040AD8B476EF20F0FC
:103EA0001550000AD8B434EF20F01550010AD8B4E8
:103EB00038EF20F01550020AD8B43CEF20F015502E
:103EC000030AD8B450EF20F01550040AD8B454EFC8
:103ED00020F01550050AD8B458EF20F01550060A06
:103EE000D8B45CEF20F01550070AD8B45FEF20F08B
:103EF0001550000AD8B463EF20F01550010AD8B469
:103F000067EF20F01550020AD8B46BEF20F015507F
:103F1000030AD8B46FEF20F01550040AD8B472EF3A
:103F200020F01550000AD8B47AEF20F01550010A9D
:103F3000D8B47EEF20F01550020AD8B482EF20F0FA
:103F40001550030AD8B486EF20F01550040AD8B4EF
:103F500076EF20F01550000AD8B490EF20F01550FD
:103F6000010AD8B494EF20F01550020AD8B498EFA3
:103F700020F01550030AD8B49CEF20F01550040A25
:103F8000D8B476EF20F01550000AD8B49DEF20F099
:103F90001550010AD8B4A1EF20F01550020AD8B488
:103FA000A5EF20F01550030AD8B4A9EF20F0155062
:103FB000040AD8B476EF20F01550000AD8B4AAEF5E
:103FC00020F01550010AD8B4AEEF20F01550020AC7
:103FD000D8B4B2EF20F01550030AD8B4B6EF20F0F1
:103FE0001550040AD8B4B7EF20F01550050AD8B41C
:103FF000BAEF20F012009E96C580152A1200E20E3C
:10400000C96E152A1200770EC96E152A1200020E0B
:10401000C96E152A12009E96C580152A1200E20E5E
:10402000C96E152A1200790EC96E152A1200000EEB
:10403000C96E152A12009E96C580152A1200E20E3E
:10404000C96E152A12007A0EC96E152A120017BC05
:1040500003D0DAC1E8FF04D01750E844E8441F0950
:10406000E8CFC9FF152A12009E96C580152A1200B6
:10407000E20EC96E152A120011BA03D011BC01D08C
:1040800003D0050E146E3ED00101D6674CEF20F030
:10409000100EC96E4EEF20F0D6C1C9FF152A1200CE
:1040A000D7C1C9FF152A1200D8C1C9FF152A1200AD
:1040B000D9C1C9FF152A1200C584152A1200FF0EA6
:1040C000156E1C9E12009E96C580152A1200E20EE7
:1040D000C96E152A1200760EC96E152A1200C58403
:1040E000152A1200FF0E156E1C9E1200C584142A9C
:1040F000156A12009E96C580152A1200E20EC96E3E
:10410000152A12007B0EC96E152A120011AA04D0BE
:10411000230EC96E152A12001C0EC96E152A120034
:104120009E96C580152A1200E20EC96E152A12004D
:104130007C0EC96E152A1200E9D79E96C580152AF5
:104140001200E20EC96E152A12007D0EC96E152AE4
:104150001200DCD79E96C580152A1200E20EC96EA9
:10416000152A12007E0EC96E152A1200CFD7C584FB
:10417000152A1200FF0E156E1C9E12001550FF0A24
:10418000D8B47CEF21F0390EC86E800EC76E280EB1
:10419000C66E000EC56E1450000AD8B4D7EF20F0DA
:1041A0001450010AD8B4EBEF20F07CEF21F0155049
:1041B000000AD8B429EF21F01550010AD8B42DEF28
:1041C00021F01550020AD8B437EF21F01550030A38
:1041D000D8B43AEF21F01550000AD8B440EF21F0DE
:1041E0001550010AD8B444EF21F01550020AD8B492
:1041F0004EEF21F01550030AD8B451EF21F01550BD
:10420000040AD8B457EF21F01550050AD8B45AEF74
:1042100021F01550060AD8B460EF21F01550070AB6
:10422000D8B463EF21F01550080AD8B469EF21F033
:104230001550090AD8B46CEF21F015500A0AD8B409
:1042400072EF21F015500B0AD8B475EF21F07CEF16
:1042500021F09E96C5807BEF21F016B004D04E0E63
:10426000C96E7BEF21F0500EC96E7BEF21F0C58443
:104270007BEF21F0142AFF0E156E12807CEF21F0E7
:104280009E96C5807BEF21F016B004D04F0EC96E0C
:104290007BEF21F0510EC96E7BEF21F0C5867BEFDD
:1042A00021F0C9CF23F0C59AC5887BEF21F0C586E0
:1042B0007BEF21F0C9CF24F0C59AC5887BEF21F0B0
:1042C000C5867BEF21F0C9CF25F0C59AC5887BEF65
:1042D00021F0C5867BEF21F0C9CF26F0C58AC588BD
:1042E0007BEF21F0C5847BEF21F0FF0E156E128667
:1042F0001C9C7CEF21F0152A120012B012D012B2D1
:1043000013D012B414D012A6120007B012001296E5
:1043100023C027F024C028F025C029F026C02AF0A9
:1043200012001290128212001292128412000001E6
:104330001550FF0A04E11294156ABEEC20F0120039
:10BF0000E844F926000C160C2B0C3F0C520C640C68
:10BF1000760C860C960CA50CB30CC10CCF0CDC0C6B
:06BF2000E80CF40C000C1B
:00000001FF
